


ARM Macro Assembler    Page 1 


    1 00000000         ;*******************************************************
                       ***********************
    2 00000000         ;* File Name          : startup_xx.s
    3 00000000         ;* Author             : SOC SA Team
    4 00000000         ;* Description        : sc32f1xxx devices vector table f
                       or MDK-ARM toolchain.
    5 00000000         ;*                      This module performs:
    6 00000000         ;*                      - Set the initial SP
    7 00000000         ;*                      - Set the initial PC == Reset_Ha
                       ndler
    8 00000000         ;*                      - Set the vector table entries w
                       ith the exceptions ISR address
    9 00000000         ;*                      - Branches to __main in the C li
                       brary (which eventually
   10 00000000         ;*                        calls main()).
   11 00000000         ;*                      After Reset the CortexM0 process
                       or is in Thread mode,
   12 00000000         ;*                      priority is Privileged, and the 
                       Stack is set to Main.
   13 00000000         ;* <<< Use Configuration Wizard in Context Menu >>>
   14 00000000         ;*******************************************************
                       *********************** 
   15 00000000         ; Amount of memory (in bytes) allocated for Stack
   16 00000000         ; Tailor this value to your application needs
   17 00000000         ; <h> Stack Configuration
   18 00000000         ;   <o> Stack Size (in Bytes) <0x0-0xFFFFFFFF:8>
   19 00000000         ; </h>
   20 00000000         
   21 00000000 00000400 
                       Stack_Size
                               EQU              0x00000400
   22 00000000         
   23 00000000                 AREA             STACK, NOINIT, READWRITE, ALIGN
=3
   24 00000000         Stack_Mem
                               SPACE            Stack_Size
   25 00000400         __initial_sp
   26 00000400         
   27 00000400         
   28 00000400         ; <h> Heap Configuration
   29 00000400         ;   <o>  Heap Size (in Bytes) <0x0-0xFFFFFFFF:8>
   30 00000400         ; </h>
   31 00000400         
   32 00000400 00000200 
                       Heap_Size
                               EQU              0x00000200
   33 00000400         
   34 00000400                 AREA             HEAP, NOINIT, READWRITE, ALIGN=
3
   35 00000000         __heap_base
   36 00000000         Heap_Mem
                               SPACE            Heap_Size
   37 00000200         __heap_limit
   38 00000200         
   39 00000200                 PRESERVE8
   40 00000200                 THUMB
   41 00000200         
   42 00000200         
   43 00000200         ; Vector Table Mapped to Address 0 at Reset



ARM Macro Assembler    Page 2 


   44 00000200                 AREA             RESET, DATA, READONLY
   45 00000000                 EXPORT           __Vectors
   46 00000000                 EXPORT           __Vectors_End
   47 00000000                 EXPORT           __Vectors_Size
   48 00000000         
   49 00000000 00000000 
                       __Vectors
                               DCD              __initial_sp ; Top of Stack
   50 00000004 00000000        DCD              Reset_Handler ; Reset Handler
   51 00000008 00000000        DCD              NMI_Handler ; NMI Handler
   52 0000000C 00000000        DCD              HardFault_Handler ; Hard Fault 
                                                            Handler
   53 00000010 00000000        DCD              MemManage_Handler 
                                                            ; MPU Fault Handler
                                                            
   54 00000014 00000000        DCD              BusFault_Handler 
                                                            ; Bus Fault Handler
                                                            
   55 00000018 00000000        DCD              UsageFault_Handler ; Usage Faul
                                                            t Handler
   56 0000001C 00000000        DCD              0           ; Reserved
   57 00000020 00000000        DCD              0           ; Reserved
   58 00000024 00000000        DCD              0           ; Reserved
   59 00000028 00000000        DCD              0           ; Reserved
   60 0000002C 00000000        DCD              SVC_Handler ; SVCall Handler
   61 00000030 00000000        DCD              DebugMon_Handler ; Debug Monito
                                                            r Handler
   62 00000034 00000000        DCD              0           ; Reserved
   63 00000038 00000000        DCD              PendSV_Handler ; PendSV Handler
                                                            
   64 0000003C 00000000        DCD              SysTick_IRQHandler 
                                                            ; SysTick Handler
   65 00000040         
   66 00000040         ; External Interrupts
   67 00000040 00000000        DCD              INT0_IRQHandler ; INT0
   68 00000044 00000000        DCD              INT1_7_IRQHandler 
                                                            ; EXTI1~EXTI17
   69 00000048 00000000        DCD              INT8_11_IRQHandler 
                                                            ; EXTI8~EXTI11
   70 0000004C 00000000        DCD              INT12_15_IRQHandler 
                                                            ; EXTI12~EXTI15
   71 00000050 00000000        DCD              RCC_IRQHandler ; RCC    ͣ    
   72 00000054 00000000        DCD              0           ; LDP
   73 00000058 00000000        DCD              BTM_IRQHandler ; BTM
   74 0000005C 00000000        DCD              UART0_2_IRQHandler 
                                                            ; UART0-UART2
   75 00000060 00000000        DCD              UART1_3_IRQHandler 
                                                            ; UART1-UART3
   76 00000064 00000000        DCD              SPI0_IRQHandler ; SPI0
   77 00000068 00000000        DCD              SPI1_IRQHandler ; SPI1
   78 0000006C 00000000        DCD              DMA0_IRQHandler ; DMA0
   79 00000070 00000000        DCD              DMA1_IRQHandler ; DMA1
   80 00000074 00000000        DCD              DMA2_IRQHandler ; DMA2
   81 00000078 00000000        DCD              DMA3_IRQHandler ; DMA3
   82 0000007C 00000000        DCD              TIMER0_IRQHandler ; TIMER0
   83 00000080 00000000        DCD              TIMER1_IRQHandler ; TIMER1
   84 00000084 00000000        DCD              TIMER2_IRQHandler ; TIMER2
   85 00000088 00000000        DCD              TIMER3_IRQHandler ; TIMER3
   86 0000008C 00000000        DCD              TIMER4_5_IRQHandler 



ARM Macro Assembler    Page 3 


                                                            ; TIMER4-TIMER5
   87 00000090 00000000        DCD              TIMER6_7_IRQHandler 
                                                            ; TIMER6-TIMER7
   88 00000094 00000000        DCD              PWM0_IRQHandler ; PWM0
   89 00000098 00000000        DCD              LEDPWM_IRQHandler ; LEDPWM
   90 0000009C 00000000        DCD              TWI0_IRQHandler ; TWI0
   91 000000A0 00000000        DCD              TWI1_IRQHandler ; TWI1
   92 000000A4 00000000        DCD              0           ; Reserved
   93 000000A8 00000000        DCD              0           ; Reserved
   94 000000AC 00000000        DCD              0           ; Reserved 
   95 000000B0 00000000        DCD              0           ; Reserved
   96 000000B4 00000000        DCD              ADC_IRQHandler ; ADC
   97 000000B8 00000000        DCD              CMP_IRQHandler ; CMP
   98 000000BC 00000000        DCD              TK_IRQHandler 
                                                            ; TK               
                                                            
   99 000000C0         
  100 000000C0         __Vectors_End
  101 000000C0         
  102 000000C0 000000C0 
                       __Vectors_Size
                               EQU              __Vectors_End - __Vectors
  103 000000C0         
  104 000000C0                 AREA             |.text|, CODE, READONLY
  105 00000000         
  106 00000000         ; Reset handler routine
  107 00000000         Reset_Handler
                               PROC
  108 00000000                 EXPORT           Reset_Handler                 [
WEAK]
  109 00000000                 IMPORT           __main
  110 00000000                 IMPORT           SystemInit
  111 00000000         
  112 00000000 481C            LDR              R0,=0x40003000
  113 00000002 6801            LDR              R1, [R0]
  114 00000004 4A1C            LDR              R2,=0x00000001
  115 00000006 4311            ORRS             R1,R1,R2
  116 00000008 6001            STR              R1,[R0]     ;AHB_CFG  开启DMA
                                                            时钟
  117 0000000A         
  118 0000000A 481C            LDR              R0,=0x4001083C
  119 0000000C 491C            LDR              R1,=0xA05F0100
  120 0000000E 6001            STR              R1,[R0]     ;DMA0_REV
  121 00000010         
  122 00000010 481C            LDR              R0,=0x4001087C
  123 00000012 491B            LDR              R1,=0xA05F0100
  124 00000014 6001            STR              R1,[R0]     ;DMA1_REV
  125 00000016         
  126 00000016 481C            LDR              R0,=0x400108BC
  127 00000018 4919            LDR              R1,=0xA05F0100
  128 0000001A 6001            STR              R1,[R0]     ;DMA2_REV
  129 0000001C         
  130 0000001C 481B            LDR              R0,=0x400108FC
  131 0000001E 4918            LDR              R1,=0xA05F0100
  132 00000020 6001            STR              R1,[R0]     ;DMA3_REV
  133 00000022         
  134 00000022 4814            LDR              R0,=0x40003000
  135 00000024 6801            LDR              R1,[R0]
  136 00000026 4A1A            LDR              R2,=0xFFFFFFFE



ARM Macro Assembler    Page 4 


  137 00000028 4011            ANDS             R1,R1,R2
  138 0000002A 6001            STR              R1,[R0]     ;AHB_CFG  关闭DMA
                                                            时钟
  139 0000002C         
  140 0000002C 4819            LDR              R0,=0x40003010
  141 0000002E 491A            LDR              R1,=0xA05F0010
  142 00000030 6001            STR              R1,[R0]
  143 00000032         
  144 00000032 481A            LDR              R0,=0x400003DC
  145 00000034 491A            LDR              R1,=0xA05F0001
  146 00000036 6001            STR              R1,[R0]
  147 00000038         
  148 00000038 481A            LDR              R0,=0X40021000
  149 0000003A 491B            LDR              R1,=0X00800000
  150 0000003C 6001            STR              R1,[R0]
  151 0000003E         
  152 0000003E 481B            LDR              R0,=0x4002105C
  153 00000040 491B            LDR              R1,=0xA05F0060
  154 00000042 6001            STR              R1,[R0]
  155 00000044         
  156 00000044 4817            LDR              R0,=0X40021000
  157 00000046 491B            LDR              R1,=0X00000000
  158 00000048 6001            STR              R1,[R0]
  159 0000004A         
  160 0000004A 481B            LDR              R0, =SystemInit
  161 0000004C 4780            BLX              R0
  162 0000004E 481B            LDR              R0, =__main
  163 00000050 4700            BX               R0
  164 00000052                 ENDP
  165 00000052         
  166 00000052         ; Dummy Exception Handlers (infinite loops which can be 
                       modified)
  167 00000052         
  168 00000052         NMI_Handler
                               PROC
  169 00000052                 EXPORT           NMI_Handler                    
[WEAK]
  170 00000052 E7FE            B                .
  171 00000054                 ENDP
  173 00000054         HardFault_Handler
                               PROC
  174 00000054                 EXPORT           HardFault_Handler              
[WEAK]
  175 00000054 E7FE            B                .
  176 00000056                 ENDP
  178 00000056         MemManage_Handler
                               PROC
  179 00000056                 EXPORT           MemManage_Handler          [WEA
K]
  180 00000056 E7FE            B                .
  181 00000058                 ENDP
  183 00000058         BusFault_Handler
                               PROC
  184 00000058                 EXPORT           BusFault_Handler           [WEA
K]
  185 00000058 E7FE            B                .
  186 0000005A                 ENDP
  188 0000005A         UsageFault_Handler
                               PROC



ARM Macro Assembler    Page 5 


  189 0000005A                 EXPORT           UsageFault_Handler         [WEA
K]
  190 0000005A E7FE            B                .
  191 0000005C                 ENDP
  192 0000005C         SVC_Handler
                               PROC
  193 0000005C                 EXPORT           SVC_Handler                    
[WEAK]
  194 0000005C E7FE            B                .
  195 0000005E                 ENDP
  197 0000005E         DebugMon_Handler
                               PROC
  198 0000005E                 EXPORT           DebugMon_Handler           [WEA
K]
  199 0000005E E7FE            B                .
  200 00000060                 ENDP
  201 00000060         PendSV_Handler
                               PROC
  202 00000060                 EXPORT           PendSV_Handler                 
[WEAK]
  203 00000060 E7FE            B                .
  204 00000062                 ENDP
  206 00000062         SysTick_IRQHandler
                               PROC
  207 00000062                 EXPORT           SysTick_IRQHandler             
   [WEAK]
  208 00000062 E7FE            B                .
  209 00000064                 ENDP
  210 00000064         
  211 00000064         Default_Handler
                               PROC
  212 00000064         
  213 00000064                 EXPORT           INT0_IRQHandler                
[WEAK]
  214 00000064                 EXPORT           INT1_7_IRQHandler              
[WEAK]
  215 00000064                 EXPORT           INT8_11_IRQHandler             
[WEAK]
  216 00000064                 EXPORT           INT12_15_IRQHandler      [WEAK]
  217 00000064                 EXPORT           RCC_IRQHandler                [
WEAK]
  218 00000064                 EXPORT           BTM_IRQHandler               [W
EAK]
  219 00000064                 EXPORT           UART0_2_IRQHandler             
 [WEAK]
  220 00000064                 EXPORT           UART1_3_IRQHandler             
[WEAK]
  221 00000064                 EXPORT           SPI0_IRQHandler          [WEAK]
  222 00000064                 EXPORT           SPI1_IRQHandler        [WEAK]
  223 00000064                 EXPORT           DMA0_IRQHandler     [WEAK]
  224 00000064                 EXPORT           DMA1_IRQHandler                
 [WEAK]
  225 00000064                 EXPORT           DMA2_IRQHandler     [WEAK]
  226 00000064                 EXPORT           DMA3_IRQHandler              [W
EAK]
  227 00000064                 EXPORT           TIMER0_IRQHandler              
 [WEAK]
  228 00000064                 EXPORT           TIMER1_IRQHandler              
 [WEAK]



ARM Macro Assembler    Page 6 


  229 00000064                 EXPORT           TIMER2_IRQHandler              
 [WEAK]
  230 00000064                 EXPORT           TIMER3_IRQHandler              
 [WEAK]
  231 00000064                 EXPORT           TIMER4_5_IRQHandler            
 [WEAK]
  232 00000064                 EXPORT           TIMER6_7_IRQHandler            
 [WEAK]
  233 00000064                 EXPORT           PWM0_IRQHandler                
[WEAK]
  234 00000064                 EXPORT           LEDPWM_IRQHandler              
 [WEAK]
  235 00000064                 EXPORT           TWI0_IRQHandler                
[WEAK]
  236 00000064                 EXPORT           TWI1_IRQHandler                
 [WEAK]
  237 00000064                 EXPORT           ADC_IRQHandler                 
 [WEAK]
  238 00000064                 EXPORT           CMP_IRQHandler                 
 [WEAK]
  239 00000064                 EXPORT           TK_IRQHandler                  
 [WEAK]
  240 00000064         
  241 00000064         INT0_IRQHandler
  242 00000064         INT1_7_IRQHandler
  243 00000064         INT8_11_IRQHandler
  244 00000064         INT12_15_IRQHandler
  245 00000064         RCC_IRQHandler
  246 00000064         BTM_IRQHandler
  247 00000064         UART0_2_IRQHandler
  248 00000064         UART1_3_IRQHandler
  249 00000064         SPI0_IRQHandler
  250 00000064         SPI1_IRQHandler
  251 00000064         DMA0_IRQHandler
  252 00000064         DMA1_IRQHandler
  253 00000064         DMA2_IRQHandler
  254 00000064         DMA3_IRQHandler
  255 00000064         TIMER0_IRQHandler
  256 00000064         TIMER1_IRQHandler
  257 00000064         TIMER2_IRQHandler
  258 00000064         TIMER3_IRQHandler
  259 00000064         TIMER4_5_IRQHandler
  260 00000064         TIMER6_7_IRQHandler
  261 00000064         PWM0_IRQHandler
  262 00000064         LEDPWM_IRQHandler
  263 00000064         TWI0_IRQHandler
  264 00000064         TWI1_IRQHandler
  265 00000064         ADC_IRQHandler
  266 00000064         CMP_IRQHandler
  267 00000064         TK_IRQHandler
  268 00000064         
  269 00000064 E7FE            B                .
  270 00000066         
  271 00000066                 ENDP
  272 00000066         
  273 00000066 00 00           ALIGN
  274 00000068         
  275 00000068         ;*******************************************************
                       ************************



ARM Macro Assembler    Page 7 


  276 00000068         ; User Stack and Heap initialization
  277 00000068         ;*******************************************************
                       ************************
  278 00000068                 IF               :DEF:__MICROLIB
  285 00000068         
  286 00000068                 IMPORT           __use_two_region_memory
  287 00000068                 EXPORT           __user_initial_stackheap
  288 00000068         
  289 00000068         __user_initial_stackheap
  290 00000068         
  291 00000068 4815            LDR              R0, =  Heap_Mem
  292 0000006A 4916            LDR              R1, =(Stack_Mem + Stack_Size)
  293 0000006C 4A16            LDR              R2, = (Heap_Mem +  Heap_Size)
  294 0000006E 4B17            LDR              R3, = Stack_Mem
  295 00000070 4770            BX               LR
  296 00000072         
  297 00000072 00 00           ALIGN
  298 00000074         
  299 00000074                 ENDIF
  300 00000074         
  301 00000074                 END
              40003000 
              00000001 
              4001083C 
              A05F0100 
              4001087C 
              400108BC 
              400108FC 
              FFFFFFFE 
              40003010 
              A05F0010 
              400003DC 
              A05F0001 
              40021000 
              00800000 
              4002105C 
              A05F0060 
              00000000 
              00000000 
              00000000 
              00000000 
              00000400 
              00000200 
              00000000 
Command Line: --debug --xref --diag_suppress=9931 --cpu=Cortex-M0+ --apcs=inter
work --depend=..\output\startup_sc32f10xx.d -o..\output\startup_sc32f10xx.o -IF
:\Users\SOC\AppData\Local\Arm\Packs\ARM\CMSIS\5.8.0\Device\ARM\ARMCM0plus\Inclu
de --predefine="__UVISION_VERSION SETA 536" --predefine="ARMCM0P SETA 1" --list
=..\list\startup_sc32f10xx.lst startup_sc32f10xx.s



ARM Macro Assembler    Page 1 Alphabetic symbol ordering
Relocatable symbols

STACK 00000000

Symbol: STACK
   Definitions
      At line 23 in file startup_sc32f10xx.s
   Uses
      None
Comment: STACK unused
Stack_Mem 00000000

Symbol: Stack_Mem
   Definitions
      At line 24 in file startup_sc32f10xx.s
   Uses
      At line 292 in file startup_sc32f10xx.s
      At line 294 in file startup_sc32f10xx.s

__initial_sp 00000400

Symbol: __initial_sp
   Definitions
      At line 25 in file startup_sc32f10xx.s
   Uses
      At line 49 in file startup_sc32f10xx.s
Comment: __initial_sp used once
3 symbols



ARM Macro Assembler    Page 1 Alphabetic symbol ordering
Relocatable symbols

HEAP 00000000

Symbol: HEAP
   Definitions
      At line 34 in file startup_sc32f10xx.s
   Uses
      None
Comment: HEAP unused
Heap_Mem 00000000

Symbol: Heap_Mem
   Definitions
      At line 36 in file startup_sc32f10xx.s
   Uses
      At line 291 in file startup_sc32f10xx.s
      At line 293 in file startup_sc32f10xx.s

__heap_base 00000000

Symbol: __heap_base
   Definitions
      At line 35 in file startup_sc32f10xx.s
   Uses
      None
Comment: __heap_base unused
__heap_limit 00000200

Symbol: __heap_limit
   Definitions
      At line 37 in file startup_sc32f10xx.s
   Uses
      None
Comment: __heap_limit unused
4 symbols



ARM Macro Assembler    Page 1 Alphabetic symbol ordering
Relocatable symbols

RESET 00000000

Symbol: RESET
   Definitions
      At line 44 in file startup_sc32f10xx.s
   Uses
      None
Comment: RESET unused
__Vectors 00000000

Symbol: __Vectors
   Definitions
      At line 49 in file startup_sc32f10xx.s
   Uses
      At line 45 in file startup_sc32f10xx.s
      At line 102 in file startup_sc32f10xx.s

__Vectors_End 000000C0

Symbol: __Vectors_End
   Definitions
      At line 100 in file startup_sc32f10xx.s
   Uses
      At line 46 in file startup_sc32f10xx.s
      At line 102 in file startup_sc32f10xx.s

3 symbols



ARM Macro Assembler    Page 1 Alphabetic symbol ordering
Relocatable symbols

.text 00000000

Symbol: .text
   Definitions
      At line 104 in file startup_sc32f10xx.s
   Uses
      None
Comment: .text unused
ADC_IRQHandler 00000064

Symbol: ADC_IRQHandler
   Definitions
      At line 265 in file startup_sc32f10xx.s
   Uses
      At line 96 in file startup_sc32f10xx.s
      At line 237 in file startup_sc32f10xx.s

BTM_IRQHandler 00000064

Symbol: BTM_IRQHandler
   Definitions
      At line 246 in file startup_sc32f10xx.s
   Uses
      At line 73 in file startup_sc32f10xx.s
      At line 218 in file startup_sc32f10xx.s

BusFault_Handler 00000058

Symbol: BusFault_Handler
   Definitions
      At line 183 in file startup_sc32f10xx.s
   Uses
      At line 54 in file startup_sc32f10xx.s
      At line 184 in file startup_sc32f10xx.s

CMP_IRQHandler 00000064

Symbol: CMP_IRQHandler
   Definitions
      At line 266 in file startup_sc32f10xx.s
   Uses
      At line 97 in file startup_sc32f10xx.s
      At line 238 in file startup_sc32f10xx.s

DMA0_IRQHandler 00000064

Symbol: DMA0_IRQHandler
   Definitions
      At line 251 in file startup_sc32f10xx.s
   Uses
      At line 78 in file startup_sc32f10xx.s
      At line 223 in file startup_sc32f10xx.s

DMA1_IRQHandler 00000064

Symbol: DMA1_IRQHandler
   Definitions
      At line 252 in file startup_sc32f10xx.s
   Uses



ARM Macro Assembler    Page 2 Alphabetic symbol ordering
Relocatable symbols

      At line 79 in file startup_sc32f10xx.s
      At line 224 in file startup_sc32f10xx.s

DMA2_IRQHandler 00000064

Symbol: DMA2_IRQHandler
   Definitions
      At line 253 in file startup_sc32f10xx.s
   Uses
      At line 80 in file startup_sc32f10xx.s
      At line 225 in file startup_sc32f10xx.s

DMA3_IRQHandler 00000064

Symbol: DMA3_IRQHandler
   Definitions
      At line 254 in file startup_sc32f10xx.s
   Uses
      At line 81 in file startup_sc32f10xx.s
      At line 226 in file startup_sc32f10xx.s

DebugMon_Handler 0000005E

Symbol: DebugMon_Handler
   Definitions
      At line 197 in file startup_sc32f10xx.s
   Uses
      At line 61 in file startup_sc32f10xx.s
      At line 198 in file startup_sc32f10xx.s

Default_Handler 00000064

Symbol: Default_Handler
   Definitions
      At line 211 in file startup_sc32f10xx.s
   Uses
      None
Comment: Default_Handler unused
HardFault_Handler 00000054

Symbol: HardFault_Handler
   Definitions
      At line 173 in file startup_sc32f10xx.s
   Uses
      At line 52 in file startup_sc32f10xx.s
      At line 174 in file startup_sc32f10xx.s

INT0_IRQHandler 00000064

Symbol: INT0_IRQHandler
   Definitions
      At line 241 in file startup_sc32f10xx.s
   Uses
      At line 67 in file startup_sc32f10xx.s
      At line 213 in file startup_sc32f10xx.s

INT12_15_IRQHandler 00000064

Symbol: INT12_15_IRQHandler



ARM Macro Assembler    Page 3 Alphabetic symbol ordering
Relocatable symbols

   Definitions
      At line 244 in file startup_sc32f10xx.s
   Uses
      At line 70 in file startup_sc32f10xx.s
      At line 216 in file startup_sc32f10xx.s

INT1_7_IRQHandler 00000064

Symbol: INT1_7_IRQHandler
   Definitions
      At line 242 in file startup_sc32f10xx.s
   Uses
      At line 68 in file startup_sc32f10xx.s
      At line 214 in file startup_sc32f10xx.s

INT8_11_IRQHandler 00000064

Symbol: INT8_11_IRQHandler
   Definitions
      At line 243 in file startup_sc32f10xx.s
   Uses
      At line 69 in file startup_sc32f10xx.s
      At line 215 in file startup_sc32f10xx.s

LEDPWM_IRQHandler 00000064

Symbol: LEDPWM_IRQHandler
   Definitions
      At line 262 in file startup_sc32f10xx.s
   Uses
      At line 89 in file startup_sc32f10xx.s
      At line 234 in file startup_sc32f10xx.s

MemManage_Handler 00000056

Symbol: MemManage_Handler
   Definitions
      At line 178 in file startup_sc32f10xx.s
   Uses
      At line 53 in file startup_sc32f10xx.s
      At line 179 in file startup_sc32f10xx.s

NMI_Handler 00000052

Symbol: NMI_Handler
   Definitions
      At line 168 in file startup_sc32f10xx.s
   Uses
      At line 51 in file startup_sc32f10xx.s
      At line 169 in file startup_sc32f10xx.s

PWM0_IRQHandler 00000064

Symbol: PWM0_IRQHandler
   Definitions
      At line 261 in file startup_sc32f10xx.s
   Uses
      At line 88 in file startup_sc32f10xx.s
      At line 233 in file startup_sc32f10xx.s



ARM Macro Assembler    Page 4 Alphabetic symbol ordering
Relocatable symbols


PendSV_Handler 00000060

Symbol: PendSV_Handler
   Definitions
      At line 201 in file startup_sc32f10xx.s
   Uses
      At line 63 in file startup_sc32f10xx.s
      At line 202 in file startup_sc32f10xx.s

RCC_IRQHandler 00000064

Symbol: RCC_IRQHandler
   Definitions
      At line 245 in file startup_sc32f10xx.s
   Uses
      At line 71 in file startup_sc32f10xx.s
      At line 217 in file startup_sc32f10xx.s

Reset_Handler 00000000

Symbol: Reset_Handler
   Definitions
      At line 107 in file startup_sc32f10xx.s
   Uses
      At line 50 in file startup_sc32f10xx.s
      At line 108 in file startup_sc32f10xx.s

SPI0_IRQHandler 00000064

Symbol: SPI0_IRQHandler
   Definitions
      At line 249 in file startup_sc32f10xx.s
   Uses
      At line 76 in file startup_sc32f10xx.s
      At line 221 in file startup_sc32f10xx.s

SPI1_IRQHandler 00000064

Symbol: SPI1_IRQHandler
   Definitions
      At line 250 in file startup_sc32f10xx.s
   Uses
      At line 77 in file startup_sc32f10xx.s
      At line 222 in file startup_sc32f10xx.s

SVC_Handler 0000005C

Symbol: SVC_Handler
   Definitions
      At line 192 in file startup_sc32f10xx.s
   Uses
      At line 60 in file startup_sc32f10xx.s
      At line 193 in file startup_sc32f10xx.s

SysTick_IRQHandler 00000062

Symbol: SysTick_IRQHandler
   Definitions



ARM Macro Assembler    Page 5 Alphabetic symbol ordering
Relocatable symbols

      At line 206 in file startup_sc32f10xx.s
   Uses
      At line 64 in file startup_sc32f10xx.s
      At line 207 in file startup_sc32f10xx.s

TIMER0_IRQHandler 00000064

Symbol: TIMER0_IRQHandler
   Definitions
      At line 255 in file startup_sc32f10xx.s
   Uses
      At line 82 in file startup_sc32f10xx.s
      At line 227 in file startup_sc32f10xx.s

TIMER1_IRQHandler 00000064

Symbol: TIMER1_IRQHandler
   Definitions
      At line 256 in file startup_sc32f10xx.s
   Uses
      At line 83 in file startup_sc32f10xx.s
      At line 228 in file startup_sc32f10xx.s

TIMER2_IRQHandler 00000064

Symbol: TIMER2_IRQHandler
   Definitions
      At line 257 in file startup_sc32f10xx.s
   Uses
      At line 84 in file startup_sc32f10xx.s
      At line 229 in file startup_sc32f10xx.s

TIMER3_IRQHandler 00000064

Symbol: TIMER3_IRQHandler
   Definitions
      At line 258 in file startup_sc32f10xx.s
   Uses
      At line 85 in file startup_sc32f10xx.s
      At line 230 in file startup_sc32f10xx.s

TIMER4_5_IRQHandler 00000064

Symbol: TIMER4_5_IRQHandler
   Definitions
      At line 259 in file startup_sc32f10xx.s
   Uses
      At line 86 in file startup_sc32f10xx.s
      At line 231 in file startup_sc32f10xx.s

TIMER6_7_IRQHandler 00000064

Symbol: TIMER6_7_IRQHandler
   Definitions
      At line 260 in file startup_sc32f10xx.s
   Uses
      At line 87 in file startup_sc32f10xx.s
      At line 232 in file startup_sc32f10xx.s




ARM Macro Assembler    Page 6 Alphabetic symbol ordering
Relocatable symbols

TK_IRQHandler 00000064

Symbol: TK_IRQHandler
   Definitions
      At line 267 in file startup_sc32f10xx.s
   Uses
      At line 98 in file startup_sc32f10xx.s
      At line 239 in file startup_sc32f10xx.s

TWI0_IRQHandler 00000064

Symbol: TWI0_IRQHandler
   Definitions
      At line 263 in file startup_sc32f10xx.s
   Uses
      At line 90 in file startup_sc32f10xx.s
      At line 235 in file startup_sc32f10xx.s

TWI1_IRQHandler 00000064

Symbol: TWI1_IRQHandler
   Definitions
      At line 264 in file startup_sc32f10xx.s
   Uses
      At line 91 in file startup_sc32f10xx.s
      At line 236 in file startup_sc32f10xx.s

UART0_2_IRQHandler 00000064

Symbol: UART0_2_IRQHandler
   Definitions
      At line 247 in file startup_sc32f10xx.s
   Uses
      At line 74 in file startup_sc32f10xx.s
      At line 219 in file startup_sc32f10xx.s

UART1_3_IRQHandler 00000064

Symbol: UART1_3_IRQHandler
   Definitions
      At line 248 in file startup_sc32f10xx.s
   Uses
      At line 75 in file startup_sc32f10xx.s
      At line 220 in file startup_sc32f10xx.s

UsageFault_Handler 0000005A

Symbol: UsageFault_Handler
   Definitions
      At line 188 in file startup_sc32f10xx.s
   Uses
      At line 55 in file startup_sc32f10xx.s
      At line 189 in file startup_sc32f10xx.s

__user_initial_stackheap 00000068

Symbol: __user_initial_stackheap
   Definitions
      At line 289 in file startup_sc32f10xx.s



ARM Macro Assembler    Page 7 Alphabetic symbol ordering
Relocatable symbols

   Uses
      At line 287 in file startup_sc32f10xx.s
Comment: __user_initial_stackheap used once
40 symbols



ARM Macro Assembler    Page 1 Alphabetic symbol ordering
Absolute symbols

Heap_Size 00000200

Symbol: Heap_Size
   Definitions
      At line 32 in file startup_sc32f10xx.s
   Uses
      At line 36 in file startup_sc32f10xx.s
      At line 293 in file startup_sc32f10xx.s

Stack_Size 00000400

Symbol: Stack_Size
   Definitions
      At line 21 in file startup_sc32f10xx.s
   Uses
      At line 24 in file startup_sc32f10xx.s
      At line 292 in file startup_sc32f10xx.s

__Vectors_Size 000000C0

Symbol: __Vectors_Size
   Definitions
      At line 102 in file startup_sc32f10xx.s
   Uses
      At line 47 in file startup_sc32f10xx.s
Comment: __Vectors_Size used once
3 symbols



ARM Macro Assembler    Page 1 Alphabetic symbol ordering
External symbols

SystemInit 00000000

Symbol: SystemInit
   Definitions
      At line 110 in file startup_sc32f10xx.s
   Uses
      At line 160 in file startup_sc32f10xx.s
Comment: SystemInit used once
__main 00000000

Symbol: __main
   Definitions
      At line 109 in file startup_sc32f10xx.s
   Uses
      At line 162 in file startup_sc32f10xx.s
Comment: __main used once
__use_two_region_memory 00000000

Symbol: __use_two_region_memory
   Definitions
      At line 286 in file startup_sc32f10xx.s
   Uses
      None
Comment: __use_two_region_memory unused
3 symbols
392 symbols in table
